:020000040000FA
:10000000000083018A010B28FD00030E8312FE000D
:100010000408FF003028F42505168B1763242218E6
:100020007324A21E0E28A212A3180E287718E1230B
:10003000F718CA23F71BB623771984238B133E22A4
:10004000221F27288B17F7197923771A6A238B1712
:10005000F71AEC23771B41235D24A21323100E28EB
:100060000C18DB228B1845280B1C83289F149F1823
:1000700037281F15231583161E088312D5001E0866
:10008000D40005080B108B1C8328231D36289F14D1
:100090009F1848281F11231183161E088312D700AA
:1000A0001E08D6009A20BC2054223E22221F692816
:1000B000DE210E2254223E22F9226A226008A80084
:1000C0006108A90070226A226208A8006308A900DA
:1000D00010235F22A216A219E8250C18DB223E226B
:1000E000221F8328771E83286A226208A5006308DE
:1000F000A6009E226008AA006108AB000E232A0811
:10010000E4002B08E50083127F0884007E0E830044
:10011000FD0E7D0E090005128E018F0105080B10E2
:100120008B1005160C10C801C7011F112311A21353
:100130002310CD29070EF039C1000E08C0000F08AA
:10014000BF000C18DB224808BE004708BD0005129E
:100150008E018F0105080B108B1005160C10C801BD
:10016000C70104300310BD0CBE0CBF0CC00CC10C89
:10017000FF3E031DB22808005508CE005408CD00EC
:100180006908CE02031CCD036808CD02CD1BD92817
:100190005508CE005408CD005908CE02031CCD03EB
:1001A0005808CD02CD1BE9285408D8005508D900BD
:1001B000E9285C08CD005D08CE005508CE02031C7E
:1001C000CD035408CD02CD1BE9285408DC005508A6
:1001D000DD005708CE005608CD006F08CE02031C84
:1001E000CD036E08CD02CD1B06295708CE00560858
:1001F000CD005B08CE02031CCD035A08CD02CD1BF7
:1002000016295608DA005708DB0016295E08CD00CB
:100210005F08CE005708CE02031CCD035608CD025E
:10022000CD1B16295608DE005708DF00FF30D00727
:10023000031CCF074F08031D08005008031D0800CA
:10024000221E24292212CD29781CCD29781D55295A
:10025000A31930298316A4038312031D5529A3155E
:10026000831620088312CD00831621088312CE0046
:100270006708CE070318CD0A6608CD070310CD0C1A
:10028000CE0C5D08CE02031CCD035C08CD02CD1F51
:100290004E29CD09CE09CE0A0319CD0A4D08031DFA
:1002A00061297608CE020318612966088316A0002A
:1002B000831267088316A10083125C08E6005D08BC
:1002C000E700781D8A29A31D8A2983162208831234
:1002D000CD00831623088312CE006D08CE070318C5
:1002E000CD0A6C08CD070310CD0CCE0C5F08CE02F2
:1002F000031CCD035E08CD02CD1F8329CD09CE0995
:10030000CE0A0319CD0A4D08031D96297608CE02A0
:10031000031896296C088316A20083126D088316B1
:10032000A30083125E08EC005F08ED005808EA00A5
:100330005908EB005A08F0005B08F1006708EB026F
:10034000031CEA036608EA026D08F102031CF003CD
:100350006C08F0026A08CD006B08CE000310CD0CCB
:10036000CE0C6708CE070318CD0A6608CD074D08E6
:10037000E8004E08E9007008CD007108CE000310B7
:10038000CD0CCE0C6D08CE070318CD0A6C08CD0736
:100390004D08EE004E08EF00A2156808D800DC00FA
:1003A0006908D900DD006E08DA00DE006F08DB00A6
:1003B000DF007408CF007508D00008005508E10080
:1003C0005408E0006708E102031CE0036608E0024D
:1003D000E01FEE29E101E001A21708009E2261085A
:1003E000AB006008AA003E22E2226A226B08A60047
:1003F0006A08A500B1222C08E1002B08E000AA0041
:100400002C08AB00AC013E220E23AA1B08003E22A2
:100410002608E1002508E000A21708005708E300BD
:100420005608E2006D08E302031CE2036C08E202D6
:10043000E21F1E2AE301E201A21708009E226308C0
:10044000AB006208AA003E22E2226A227108A600DE
:100450007008A500B1222C08E3002B08E200AA00D6
:100460002C08AB00AC013E220E23AA1B08003E2242
:100470002608E3002508E200A21708006A222213DA
:100480007208A500031D22177308A600031D22177A
:1004900008002A08A5002B08A6002C08A7002D0894
:1004A000A8002E08A90008004108AE004008AD00D1
:1004B0003F08AC003E08AB003D08AA0008002E082B
:1004C000C6002D08C5002C08C4002B08C3002A084C
:1004D000C2000800A501A601A701A801A901080002
:1004E0002908AE07031883222808AD0703188522C0
:1004F0002708AC07031887222608AB070318AA0AA7
:100500002508AA070800AD0A0319AC0A0319AB0AAB
:100510000319AA0A0800A709A609A509982AA90982
:10052000A809A709A609A509A90A0319A80A031970
:10053000A70A0319A60A0319A50A0800AA01AB0114
:10054000AC01AD01AE010800AC09AB09AA09852ACE
:10055000AE09AD09AC09AB09AA09AE0A0319832A91
:1005600008001830D100CE01CD010310AC0DAB0D49
:10057000AA0DCE0DCD0D4E08A9004D08A8002213DE
:100580002608CE020318C82AFF30CD07031C221705
:100590002508CD02031C22170310221F0314221F5B
:1005A000D52A2908CE002808CD00D10BB62AAC0DDB
:1005B000AB0DAA0D08000C10C80A0319C70A0319CD
:1005C000231408002508CD002608CE006A222A0838
:1005D000A6002B08A7009E221030D1000310AC0DFE
:1005E000AB0DAA0DCE0DCD0D03187822D10BEE2A3E
:1005F00008002508CD002608CE0049229E22103092
:10060000D1000310AE0DAD0DAC0DAB0DAA0DCE0D8E
:10061000CD0D03187022D10B012B08008B22782AF4
:100620008F22702A6608B9006708BA00522368084A
:10063000B9006908BA0052236A08B9006B08BA0009
:1006400052236C08B9006D08BA0052236E08B90035
:100650006F08BA0052237008B9007108BA00522B13
:100660007208B9007308BA00522B4430781945302B
:1006700059247608BA00582B7408B9007508BA00D6
:100680004F2BBA010830F818BA0704307818BA07A7
:1006900002302318BA070130A21BBA07582B390EB3
:1006A000A0005C233908A0005C233A0EA0005C2364
:1006B0003A08A0005C23612C20080F39093C20086F
:1006C0000F39031C073E303E592C7208B8007308DE
:1006D000B900D32B6408B8006508B9002030B81FF2
:1006E000772BB809B909B90A0319B80A2D3059246A
:1006F000D32B6008B8006108B900D3236208B800A2
:100700006308B900D32BCA236608B8006708B9008C
:10071000D3236A08B8006B08B900D3236C08B8006B
:100720006D08B900D3237008B8007108B900D32B45
:100730006608B8006708B900D3236808B8006908DC
:10074000B900D3236A08B8006B08B900D3236C083A
:10075000B8006D08B900D3236E08B8006F08B9005F
:10076000D3237008B8007108B900D32B5C08B80017
:100770005D08B900D3235808B8005908B900D3233D
:100780005E08B8005F08B900D3235A08B8005B08B8
:10079000B900D32B5408B8005508B900D323560824
:1007A000B8005708B90003243608A00056244C248A
:1007B000612C7408B8007508B900032443244C2444
:1007C000612C3D08B8003E08B9003F08BA00400857
:1007D000BB004108BC00F62B4608BC004508BB0026
:1007E0004408BA004308B9004208B8001424370886
:1007F000031D23143608031D23144C244E245024B7
:1008000052245424612C03101030AF002C24B90D55
:10081000B80DB50DB60DB70DAF0B0F2C0800353068
:10082000840003303424072C03102830AF002C241C
:10083000BC0DBB0DBA0DB90DB80DB10DB20DB30D98
:10084000B40DB50DB60DB70DAF0B272C0800313028
:10085000840007303424182CB701B601B501B40167
:10086000B301B201B1010800C9000008033EB000A5
:10087000B01980000008303EB000B01B8000840A30
:10088000C90B352C08003708A00056243608A000F4
:10089000A00E5624A00E562C3508472C3408472CA1
:1008A0003308472C3208472C3108472C20080F39D1
:1008B000303E961C592C950008000D3059240A3002
:1008C000592C2030592C8C1E080017080639031D9E
:1008D0006D2C1408A1002214080017121408171612
:1008E0002210A401080022102330A525031D7C2C12
:1008F0002211A210D301A32DA41F822CB5252219E9
:100900000800A32D241FA42C6330A525031D8B2CC8
:100910009823D923A22C6730A525031D912C65238C
:10092000A22C6930A525031D972C8323A22C73309C
:10093000A525031D9D2C4123A22C7430A525031D44
:10094000A32DD9235D24A32DA41EDF2C6330A52560
:10095000031DAD2C7708043ADD2C6430A525031D5A
:10096000B42C7708203ADD2C6930A525031DBB2C5B
:100970007708083ADD2C7030A525031DC22C7708B6
:10098000803ADD2C7230A525031DC92C7708023A68
:10099000DD2C7330A525031DD02C7708403ADD2CC3
:1009A0007430A525031DD72C7708013ADD2C76304D
:1009B000A525031DA32D7708103AF700A32D241EAB
:1009C0002F2D6430A525031DE72C7810A32D65304D
:1009D000A525031DEE2C7814CD21A32D6730A52568
:1009E000031DF52CA21472305C2D6930A525031D62
:1009F000FD2CF8141116A215A32D6C30A525031D8E
:100A0000032D7815A32D6E30A525031D0B2DF81091
:100A10001112A215A32D7030A525031D142D12232C
:100A200030233C233523A22C7230A525031D1A2D1B
:100A3000CD21A32D7430A525031D202D74305C2DF0
:100A40007530A525031D262D7811A32D7630A525FB
:100A5000031DA32DA2147630CC0001305E2DA41D01
:100A6000462D6330A525031D382DA2146E305C2D54
:100A70007330A525031D3F2DA21470305C2D7A30F4
:100A8000A525031DA32DA2146C305C2D241D632D00
:100A90006330A525031D4F2DA21468305C2D7330E3
:100AA000A525031D562DA2146A305C2D7A30A5258C
:100AB000031DA32DA2146630CC000230CB00D3015D
:100AC0002215A4170800A41C962D4130A525031D4E
:100AD0006B2D241508004230A525031D712DA4158A
:100AE00008004330A525031D772D24160800443047
:100AF000A525031D7D2DA41608005030A525031D36
:100B0000832D241708005230A525031D8A2DA3101C
:100B10008B20A32D5330A525031D902DA314A32DA9
:100B20005530A525031DA32DA215A32D4030A525C5
:100B300003199D2D2418241008002418A12D241415
:100B40000800A4140800A4010800C90021084902F3
:100B500008002108C900491FB02DC9120730C90279
:100B60003030C90249080F390800A925A218BC2D48
:100B7000D300D30EA2140800D3074C0884005308F6
:100B80008000D301A210CB0BC72D22110800840ACC
:100B90000408CC0008005208031383169B009C1322
:100BA0001C141A08831208000008031383169A0005
:100BB0008312520883169B009C131C1555309D0010
:100BC000AA309D009C141C119C18E42D831208006F
:100BD000A211D201663084001330D100D425D20A8C
:100BE000840AD10BEE2D0800850187018B0190014D
:100BF000073099009A106400831671308F004730D7
:100C000081000330910050309F002F3085003F302D
:100C1000870001308C0008309600831281309F00DD
:100C200096161615333093001112171697170630C3
:100C300090008E018F01C701C8018C010B170B16A4
:100C40008B15A201A301A4010301D2006630840028
:100C50001330D100CB258000D20A840AD10B2A2E72
:100C6000F81811166808D800DC006908D900DD0002
:100C70006E08DA00DE006F08DB00DF000130CF0015
:100C80002C30D000221604308316A4008312A31146
:100C90001F11231105080B100800500049004300E4
:100CA000540049004300200049004900200056003C
:100CB00065007200200031002E00300030002C0052
:100CC000200043006F007000790072006900670027
:100CD000680074002000A900200052006900630031
:100CE00068006100720064002000480020004D0090
:100CF000630043006F0072006B006C006500200011
:0A0D00003200300031003000200006
:02400E00C430BC
:00000001FF
